:020000040000FA
:040000006C303A28FE
:08000800A000030EA100831209
:1000100005191028831601178312B23081002B288E
:1000200083160113831203140B190310A80DA90DD5
:10003000AA0DAB0DAC0DAC16FF302C02031D2B2806
:10004000FA302B02031D2B2831152A08AF0029088E
:10005000AE002808AD008B100B11210E8300A00EFE
:04006000200E090065
:0C007400203084008001840A6030040207
:10008000031C3C281230B000922183160C308505E9
:1000900087018312850187010730990000309A009B
:1000A000103083168E008312603083168F00831207
:1000B0000030831691008312C830831681008312AA
:1000C00031309000003083168C00831210308B008A
:1000D000831600309B001C141A088312BC00851D77
:1000E000D621831610309B001C141A088312BD0001
:1000F000CE2181018E018F010B118B100B108C0111
:100100008B17902031199320B30B8E28031085197B
:100110000314B90DF030390203190F21FB21812896
:1001200064003210080031110130B7008B13203009
:10013000370783169B001C141A088312A400103082
:10014000370783169B001C141A088312A300A6000D
:100150000230A6060030370783169B001C141A08CD
:100160008312A200A7000130A7068B17321CBE28FD
:1001700022090339A200A309A409A50924082F0212
:10018000031D092923082E02031D092922082D0217
:10019000031D092901303702031DD3283D18D32838
:1001A0003D143E149E2102303702031DDC28BD1889
:1001B000DC28BD143E14A02103303702031DE528BE
:1001C0003D19E5283D153E14A22104303702031DD8
:1001D000EE28BD19EE28BD153E14A42105303702C6
:1001E000031DF7283D1AF7283D163E14A6210630B8
:1001F0003702031D0029BD1A0029BD163E14A8218F
:1002000007303702031D09293D1B09293D173E14FC
:10021000AA21B70A083037020318080096280130CF
:10022000B600B300B400B500B70085018701B11373
:100230009020B30B4329031085190314B90DF03036
:10024000390203196A29B40B432901303702031913
:10025000B521023037020319BA21033037020319DE
:10026000BD21043037020319C021053037020319BC
:10027000C521063037020319C82107303702031998
:10028000CB219630B400311D18293111321C4D2973
:100290002D090339AD00AE09AF092F1C18298E01B5
:1002A0008F010C1C18290C102E1E18298B132030BE
:1002B0003707BB002F08BA007D2110303707BB007D
:1002C0002E08BA007D2100303707BB002D08BA0088
:1002D0007D218B1785018701B70AB60108303702E7
:1002E000031C1829CE2108003E1C08003E101030C7
:1002F000BB003D08BA007D2108008B133A08831625
:100300001C159A0083123B0883169B0055309D00F4
:10031000AA309D009C1464009C188B291C11831228
:100320008B170800FF30D000D415D515D615D7157A
:10033000D815D915DA15DB15DC150800F130AD2913
:10034000F230AD29F430AD29F830AD291F30B12994
:100350002F30B1294F30B1290800BD050F30D2042C
:100360000800BD05F030D2040800103085060230C8
:100370008706080020308506080021308506080021
:10038000023085060230870608001830870608000C
:100390002130870608000930870608003D08D20092
:1003A000031D08001130BD00D2000800B601B301E2
:1003B000B4013C1CDE29BC01BC14E029BC013C1486
:1003C0003C08B6006400E429E529E629E729E82984
:1003D000B41B0516B41F0512B30BE229B40BE229B6
:1003E0000310B60CB608031DE2290030BB003C0820
:1003F000BA007D2108008F08031908008F01D00F73
:10040000362BD00A0E305205031D152A541D0B2A17
:10041000D4015416232AD41D102AD4015416232A99
:10042000541E232AD401D414232AD41C1A2AD401FA
:100430005415232A541D1F2AD401D415232A541ECF
:10044000232AD401541509305205031D362A551D9F
:100450002C2AD5015516442AD51D312AD501551609
:10046000442A551E442AD501D514442AD51C3B2ABA
:10047000D5015515442A551D402AD501D515442AC4
:10048000551E442AD50155150B305205031D572A18
:10049000561D4D2AD6015616652AD61D522AD6015A
:1004A0005616652A561E652AD601D614652AD61C0C
:1004B0005C2AD6015615652A561D612AD601D61525
:1004C000652A561E652AD601561507305205031DAA
:1004D000782A571D6E2AD7015716862AD71D732AE8
:1004E000D7015716862A571E862AD701D714862A7F
:1004F000D71C7D2AD7015715862A571D822AD70176
:10050000D715862A571E862AD70157150630520559
:10051000031D992A581D8F2AD8015816A72AD81DBD
:10052000942AD8015816A72A581EA72AD801D814E9
:10053000A72AD81C9E2AD8015815A72A581DA32AD5
:10054000D801D815A72A581EA72AD8015815103047
:10055000BC1819305205031DBC2A591DB22AD901F5
:100560005916CA2AD91DB72AD9015916CA2A591E9D
:10057000CA2AD901D914CA2AD91CC12AD9015915A4
:10058000CA2A591DC62AD901D915CA2A591ECA2AEA
:10059000D90159155030BC1859305205031DDF2AB6
:1005A0005A1DD52ADA015A16ED2ADA1DDA2ADA019D
:1005B0005A16ED2A5A1EED2ADA01DA14ED2ADA1C4F
:1005C000E42ADA015A15ED2A5A1DE92ADA01DA1568
:1005D000ED2A5A1EED2ADA015A156030BC1869302E
:1005E0005205031D022B5B1DF82ADB015B16102B45
:1005F000DB1DFD2ADB015B16102B5B1E102BDB01C4
:10060000DB14102BDB1C072BDB015B15102B5B1D98
:100610000C2BDB01DB15102B5B1E102BDB015B159C
:100620002030BC1829305205031D252B5C1D1B2BC7
:10063000DC015C16332BDC1D202BDC015C16332B1C
:100640005C1E332BDC01DC14332BDC1C2A2BDC017D
:100650005C15332B5C1D2F2BDC01DC15332B5C1E52
:10066000332BDC015C1574213D08D2005008D10009
:100670000C305405031D05120C305505031D851261
:100680000C305605031D05100C305705031D851051
:100690000C305805031D87100C305905031D071039
:1006A0000C305A05031D87120C305B05031D071221
:1006B0000C305C05031D871151080E020318882BAE
:1006C00012305405031D051612305505031D8516FD
:1006D00012305605031D051412305705031D8514ED
:1006E00012305805031D871412305905031D0714D5
:1006F00012305A05031D871612305B05031D0716BD
:1007000012305C05031D8715FF30500203190800E5
:100710008F08031D0800902051080E02031C882B2F
:1007200018305405031D051206305405031D051627
:1007300018305505031D851206305505031D851615
:1007400018305605031D051006305605031D051407
:1007500018305705031D851006305705031D8514F5
:1007600018305805031D871006305805031D8714DF
:1007700018305905031D071006305905031D0714CD
:1007800018305A05031D871206305A05031D8716B7
:1007900018305B05031D071206305B05031D0716A5
:1007A00018305C05031D871106305C05031D871595
:0207B00008003F
:084000000A00030002000600A3
:02400E00CC33B1
:10420000010078007A007C007E007B0079007F004E
:104210007D007A0078007E007C00FF00FF00FF0038
:104220000000F200F600FA00FE00F200F600FA00CC
:10423000FE00F200F600FA00FE00FF00FF00FF00A3
:10424000010005000500050005000900090009003E
:1042500009000D000D000D000D00FF00FF00FF0024
:10426000FF00FF00FF00FF00FF00FF00FF00FF0056
:10427000FF00FF00FF00FF00FF00FF00FF00FF0046
:10428000FF00FF00FF00FF00FF00FF00FF00FF0036
:10429000FF00FF00FF00FF00FF00FF00FF00FF0026
:1042A000FF00FF00FF00FF00FF00FF00FF00FF0016
:1042B000FF00FF00FF00FF00FF00FF00FF00FF0006
:1042C000FF00FF00FF00FF00FF00FF00FF00FF00F6
:1042D000FF00FF00FF00FF00FF00FF00FF00FF00E6
:1042E000FF00FF00FF00FF00FF00FF00FF00FF00D6
:1042F000FF00FF00FF00FF00FF00FF00FF00DD00E8
:00000001FF
